:030000000219FDE5
:03000B000200A848
:03002B0002015A75
:03005B000202EEB0
:030073000202DBAB
:1000800002030406080C10182030406080040608A3
:100090000C10182030406080A0C00003070F1F051F
:1000A000050D050305030302C2AFC0D0C0E0206206
:1000B00014E5256009E473E525F4F58AD262D0E001
:1000C000D0D0D2AF3285268AC262E526F4602F30C6
:1000D000682520720DD0E0D0D0C293C295C297D2CD
:1000E000AF32C293C295C297206F0C206609740A82
:1000F000D5E0FDE57B4290D0E0D0D0D2AF32758A1A
:1001000000C28DD26201F701B7306805206602D2C5
:100110009301B7306805206602D29501B7306805B3
:10012000206602D29701B7C29230680A206607742F
:1001300008D5E0FDD29301B7C29430680A20660763
:100140007408D5E0FDD29501B7C29630680A2066E2
:10015000077408D5E0FDD29701B7C2AFC2AD53E630
:10016000EFC0D0C0E0D2D3D2AFC2CEE52A60072024
:100170007449152A21BB7800790020742EE580305F
:100180007E01F430E30278FF53DACF207E0343DAB6
:1001900020307E0343DA10C2D8C271E580307E0180
:1001A000F430E30279FFC3E89970CB306103752A1C
:1001B00018207403752A18885CD27020740DE52B02
:1001C0006004152B21CB43DA01C2D8207002413ED6
:1001D000A85C206102C270207431C3E894F040032F
:1001E00074F0F8E8C4540F28F87984B70302410B7F
:1001F000C313C3138721200802C313200A06C3C8F0
:1002000098F8410B28F8500374FFF8C3E89565503F
:1002100003E565F88822E52D54066022206B1FE572
:1002200036C333C333F8E564C313C313F9C395224C
:1002300040028922E82522F52250037522FF8522FB
:1002400024A824C3E52495614002A8618825E566B9
:1002500070024182C3E8AA669A5003E8FAE4F9EA18
:10026000C333FBE568F45B29400D2567F8E567605B
:10027000021567400B41820AC3E5679A5002056781
:1002800078FF8826C26FC3E52694F84002D26FC378
:10029000E52594404002D26420CF0AD0E0D0D0437C
:1002A000E610D2AD32C2CF053A7801E52A600530BA
:1002B0007402152AC3E55C94014005755F0041D1C5
:1002C000756000756900E55F2401F55F5003755F97
:1002D000FFD0E0D0D043E610D2AD32C2AF53E67FBC
:1002E0007592FA7593FFC260759104D2AF32C2AFB6
:1002F00053E6EFC2ADC0D0C0E0C0F0D2D3D2AFA8B9
:10030000FBA9FCC2D8307102615553DACF207E03BD
:1003100043DA10307E0343DA20D271E580307E016B
:10032000F420E302612C88278928A18253DACF20A8
:100330007E0343DA20307E0343DA10C2D8C2713024
:100340007402A16E7800E580307E01F430E302A1F2
:100350006E885CA15653DACF207E0343DA20307ECC
:100360000343DA10C271206102812E53DACF207E5E
:100370000343DA10307E0343DA20C2D8D2718857A3
:100380008958C3E89555F8E99556F97B007E087AB7
:1003900000C3E8948CE994005005755B00812088C7
:1003A0002178A2E6A8216055C3E894C8E9940050DA
:1003B00008E4D2E4FB7A0A61FBC3E89468E994019B
:1003C0005008E4D2E3FB7A0F61FBC3E894D0E994D0
:1003D000025008E4D2E2FB7A1E61FBC3E894A0E974
:1003E00094055008E4D2E1FB7A3C61FBC3E89498A1
:1003F000E994085008E4D2E0FB7A787E00C3E895DF
:1004000059FCE9955AFD30E70AECF42401FCEDF4BF
:100410003400FD755B00C3EC9AED9E5003755B01E3
:100420008859895A8557558558567802A156C3E888
:100430009527F8E99528F9307C02A13A307B02A192
:100440003A307A02A1332075028151E9FDE8FC813E
:1004500070E9C313F9E813F8307902A133E9C31343
:10046000F9E813F8307802A133E9C313FDE813FC6F
:0F04700020612CC3EC941CED940240028187EDB7
:10047F00701EC3EC94C850180529E5297002152980
:10048F00C3E529940A5002A16E755C00D270A16E6B
:10049F00E529600215297888E6F97400207F08782D
:1004AF0096B90302789EE624FAFEE43400FFC3EC0B
:1004BF009EFCED9FFD9208B90310A208500720760D
:1004CF0009D27681D9307602C276A2085016B903C6
:1004DF000DECF42401FCEDF43400FD0204F378007C
:1004EF007900A13AB90315EC33FCED33FDC3EC945D
:1004FF000AFCED9400FD50047C007D00C3EC94FFDA
:10050F00ED9400400678FF7900A13AEC8572F0A4D3
:10051F00C5F0A2F733F87900400302055678FF794A
:10052F0000020556E9C313F9E813F8307C0EE960B1
:10053F000278FFC3E81338F8E43400F9C3E894FFF6
:10054F00E99400400278FF885CD270206102A16EAE
:10055F00741FF4552F4BF52FC274EB7002D27475C4
:10056F002A18307403752A0A306102A1822074039D
:10057F0053DAFE207403752B06D0F0D0E0D0D0D222
:10058F00AD43E6103279010205B279030205B27963
:10059F000A0205B2791E0205B279640205B279C862
:1005AF000205B27817E4D5E0FDD8FAD9F6227A140D
:1005BF007B780205D97A107B8C0205D97A0D7BB432
:1005CF000205D97A0B7BC80205D97902E4C294D50A
:1005DF00E0FDD295D5E0FDC295D5E0FDD294D5E0F2
:1005EF00FDE920E002D29330E002D297E573D5E027
:1005FF00FDE920E002C29330E002C2977496D5E085
:10060F00FDD9C9EAF8D5E0FDD8FBDBBEC29422C301
:10061F007C007D0075F00005F0EA33FAEB33FB50F8
:10062F00F6EB13FBEA13FAC3E9FFE8FEE89AF8E9E1
:10063F009BF95004EFF9EEF8B3EC33FCED33FDD535
:10064F00F0DFEDF9ECF822E889F08A20D2D4F8A98E
:10065F00F07B0030F70B7BFFF42401F8E9F4340052
:10066F00F9E88520F0A4ADF0F8E98520F0A4AFF00B
:10067F00FEED2EF974003FFA7C04C3EA13FAE91376
:10068F00F9E813F8DCF48BF030F70AE8F42401F8FA
:10069F00E9F43400F9E889F0C2D4F8A9F02222C3B2
:1006AF00E54113F9E54013F8C3E54498F8E545999A
:1006BF00F9500CC3E89480E994FF40160206E5C395
:1006CF00E8947FE9940050030206E5787F790002F1
:1006DF0006E5788079FF8849894A22E5492546F859
:1006EF00E54A3547F9854A20E4300701F43548FAE1
:1006FF0030E709C3EA94F04015020723C3EA940FC9
:10070F00500302072378FF79FF7A0F02072378003F
:10071F0079007AF0C3E5249561500AC374019524DA
:10072F00500B020741E54A20E70E020741E54A3028
:10073F00E706884689478A482278A5E6FAC3E5493D
:10074F0033F8E54A33F9D156E930E70BC3E8948023
:10075F00E994FF4013E17BC3E8947FE994005002D2
:10076F00E17B787F7900E17B788079FFE820E715DE
:10077F00C3E52398F84009C3E8940140030207A298
:10078F0078010207A2E8F424012523F840030207A9
:10079F00A278FF884B2278A6E6FAA847A948D15637
:1007AF00E930E70CC3E89401E994FF40160207D63D
:1007BF00C3E894FFE9940050030207D678FF79004D
:1007CF000207D6780179FFE920E715C3E54B98F8C2
:1007DF004009C3E8940140030207FD78010207FDB9
:1007EF00E8F42401254BF840030207FD78FF882425
:1007FF002278FFC26420693D206A12D264C3E541AA
:10080F00940A4009C3E52594405002C26479A1E7D8
:10081F006023E541601F74FF8541F0848539F03016
:10082F006A0375F005A4F8C5F0600278FFC3E89578
:10083F00645002A864886322C3E5409440E5419464
:10084F0001E5635003140158046002F563220208A6
:10085F00602275E890227883E6FFE5E820ECF7A8A0
:0F086F00BDA9BE0570C3E57094084052757000B6
:10087E00E9FA79A0E76044EA7007E571601B0208A7
:10088E009BC3E895716010E5715006600C14020868
:10089E00A70460F90208A7E571F571C394A8401B7F
:1008AE007561C0C394054013756180C39405400BF8
:1008BE00756140C39405400375610075BB0122E567
:1008CE0061F460020561E570B4070375BB1E227406
:1008DE003279A787F0A4C5F0A2F733F8C3E8956183
:1008EE004002A8618822882488258826886422757B
:1008FE0040007541F022C2AF75C820A8CCA9CDAA80
:10090E003A30CF010A75C824D2AFAB3BAC3C883B22
:10091E00893CC3E89BF8E99C206908F930670241DD
:10092E0010216DAD3D8A3DF9EA9DFA600478FF799C
:10093E00FFAE3EAF3F8B3E8C3FA83BA93CC3E89E2B
:10094E00F8E99FF9C3E54113FBE54013FAE82AF5F0
:10095E0040E93BF54150067540FF7541FF21B7AAAE
:10096E0040AB41AC40AD417E047F02C3EB940440EA
:10097E00021E1FC3EB940840021E1FC3ED13FDECB5
:10098E0013FCDEF7C3EA9CFAEB9DFBEF6009C3E9AB
:10099E0013F9E813F8DFF7EA28FAEB39FB8A408BF4
:1009AE004150067BFF8B408B41C3EB94025002D229
:1009BE00673069047F0321E27892E6FFC3E537943E
:1009CE008240110FC3E53794A040010FC3EF940688
:1009DE0040027F057E02E541C4540FF9E541C4543F
:1009EE00F0F8E540C4540F28F8C3E89EFAE99400E5
:1009FE00FB4009C3EA9402EB940050047A02E4FB34
:100A0E00415CAA40AB41EBC4FEEAC4540F4EFCC39A
:100A1E00EA9CFAEB9400FBC3E813C313F8EA28FA36
:100A2E00EB3400FB8A408B41C3EB94024002C26759
:100A3E007802EBC4FE7B00EAC4540F4EFAC3EA9868
:100A4E00FA4005C3940250027A027892E6FF3060B3
:100A5E0002415C855192855293D26043E680C3E495
:100A6E009AF8E49BF930670241E8E8FAE9FBD3E92A
:100A7E0013FDE813FC88518952C3EF94036038EFDD
:100A8E0020E00DE82CF8E93DF9ECFAEDFB020AB195
:100A9E00E828F8E939F9C3E82402F8E93400F97ACC
:100AAE00FE7BFFC3EF9403400E8A538B54884D890F
:100ABE004E8C4F8D50611C885389548A4D8B4E8CB1
:100ACE004F8D503069127553F07554FF754FF07598
:100ADE0050FF7551F07552FF611CE8FAD3E813FC14
:100AEE008851C3EF94036020EF20E007E82CF8EC68
:100AFE00FA6108E8282402F87AFEC3EF940340084E
:100B0E008A53884D8C4F611C88538A4D8C4FE568F3
:100B1E00C3335002646BF56830600261267534028F
:100B2E00D26043E680E52D54066034A840A941C347
:100B3E00E913F9E813F8C3E913F9E813F830690477
:100B4E00E92440F9C2AF53E67F759100C3E498F5EE
:100B5E0094E499F595759104D26043E680D2AF2264
:100B6E00D265754300752000306C03752040020B72
:100B7E008DD265754300752040306C03752000786A
:100B8E00017901206720E52D54066002C2657914B3
:100B9E00E541C313700104F8C39414400278143075
:100BAE006904781B791B206010E543600C306903E3
:100BBE00D53404D26D8138712E0543E59E7005E55E
:100BCE009B020BD4E59A5440B5200281223069096C
:100BDE0008C3E89940011861B420650A08C3E89972
:100BEE004002618D61B4C265C2AF53E67F7591005C
:100BFE003067127594007595FE759104D26043E6C8
:100C0E0080D2AF618DAE40AF41C3E49EF594E49FB8
:100C1E00F5958107C3E53394015002618D3065026D
:100C2E00618DD802813661B4C26DC2AF53E67F7555
:100C3E009100855394855495759104854D92854EFA
:100C4E0093D26043E680D2AFE52D54066008206A49
:100C5E00020533020C74306D0D206C0A20650715E9
:0F0C6E0081158102153922780030640530650246
:100C7D007801E53775F007A4F9E5F028F5F0E9A25C
:100C8D00F013A2F113A2F213F537C3947850037544
:100C9D003778C3E53795384008D266C293C295C2FE
:100CAD009730600281AE854F92855093D26043E6B6
:100CBD008022207D19C2AF754202C294D292306259
:100CCD0002D297D2AF759F33759E00020EC0C2AF90
:100CDD00754202C294D296306202D293D2AF759F02
:100CED0033759E00020EC0307243207D20C2AF7559
:100CFD004203900138757B10C297C296306204D2C0
:100D0D0095A112D294D2AF759E23020EC0C2AF75BB
:100D1D004203900138757B10C293C292306204D2A7
:100D2D0095A132D294D2AF759E22020EC0207D17AE
:100D3D00C2AF754203900113C297306202D295D2B1
:100D4D00AF759E23020EC0C2AF754203900113C250
:100D5D0093306202D295D2AF759E22020EC0207DD5
:100D6D0016C2AF754204C292D296306202D295D2AB
:100D7D00AF759E22020EC0C2AF754204C296D292CA
:100D8D00306202D295D2AF759E23020EC0307249E9
:100D9D00207D23C2AF754205900127757B04C29556
:100DAD00C294306204D293A1B8D292D2AF759F3360
:100DBD00759E00020EC0C2AF754205900149757B4C
:100DCD0040C295C294306204D297A1DBD296D2AFC5
:100DDD00759F33759E00020EC0207D1AC2AF7542FD
:100DED0005900109C295306202D293D2AF759F333F
:100DFD00759E00020EC0C2AF75420590011DC295D1
:100E0D003062E8D297D2AF759F33759E00020EC047
:100E1D00207D16C2AF754206C296D294306202D2C0
:100E2D0093D2AF759E23020EC0C2AF754206C29219
:100E3D00D294306202D297D2AF759E22020EC0308C
:100E4D007243207D20C2AF754201900149757B40F0
:100E5D00C293C292306204D297C16AD296D2AF7554
:100E6D009E22020EC0C2AF754201900127757B0410
:100E7D00C297C296306204D293C18AD292D2AF7514
:100E8D009E23020EC0207D17C2AF75420190011D39
:100E9D00C293306202D297D2AF759E22020EC0C2AB
:100EAD00AF754201900109C297306202D293D2AF61
:100EBD00759E23C26622900107757B00C293C29571
:100ECD00C297C292C294C296C26222788076FF08FF
:100EDD0076FF0876FF0876FF087603087604087615
:100EED0007087603087601087601788C7601087676
:100EFD00FF0876FF0876FF0876FF0876FF08760371
:100F0D000876FF0876FF0876FF0876250876D00864
:100F1D0076FA0876FA0876040876FF0876010876E0
:100F2D000008767A0876FF087601087601087600C3
:100F3D00087603087600227887E6FFC272BF0302A7
:100F4D00D2727888E6C394036008C27DE630E10270
:100F5D00D27DC27E7889E630E102D27EC3EF940263
:100F6D006008758E01D273020F7C758E00C27322DC
:100F7D007880E6149000809378A5F67881E6149039
:100F8D0000809378A6F67886E61490008D9378A766
:100F9D00F67886E6F539C394025003753902789CCC
:100FAD00E67538FFB402037538A0B40303753882B3
:100FBD0078A3E61490009A93F566D1C32222789611
:100FCD00E6FA7897E6FB7888E6B40305C3EB940E52
:100FDD00FB307F047A007BFFC3EB9AFCC3948250F5
:100FED00027C827572000572EC8572F0A4C3E5F087
:100FFD00947D40F222D27F120FCB1205A37A007B93
:10100D00007C10120599E55C2AFA74003BFBDCF3B9
:10101D007C04C3EB13FBEA13FADCF7FEC27F120F5D
:10102D00CB22E5EF20E6037520000520903DFFE57E
:10103D0020146006901FFF1460009304600375EF89
:10104D001253D9BF7581C043FF8012059475EF020D
:10105D0043B203E5B3240220E70DF521E5B120E00D
:0D106D00068521B343B101120EC375800842
:10107A0075A40075F1FF75D4F775900275A5FC7516
:10108A00F2FC75D50075A0FD75A60275F30275D63A
:10109A000075B0FF75A70175F4FF75E241120EC322
:1010AA00E4F8F6D8FD756801120ED812158A7898F8
:1010BA008673753001C2AF1205AD1205BD1205A3C4
:1010CA001205C41205A31205CB1205A31216A31208
:1010DA0005AD1205AD1205A8C2AF78FA79FA3083C8
:1010EA0007D9FBD8F7021C00120F44120F7D120F0A
:1010FA00CA120FCB78988673120EC3758810758939
:10110A000275C82475910475D84075A82275B8026D
:10111A0075E690759B80759D00759A80759C007523
:10112A00D10E75BC5875BB0175BA1F75E8801205DA
:10113A0094D2AF12085D75360053DACF207E03438E
:10114A00DA20307E0343DA1043DA01C2D8C27112C0
:10115A0005ADD2617B037A0CE55B70077A0CDB0381
:10116A000210E21205A32070030210E2C270E55CCD
:10117A00C3940240E1E52F541F855E5DF55EB55DBF
:10118A00D5DAD5C26153DACF207E0343DA20307E26
:10119A000343DA10C2D8C27178A2E67008D274E5A5
:1011AA002F54E0F52FC2757529001205A83074096D
:1011BA00C3E529940A4002D275120599780230745F
:1011CA00027800C3E55C9840F0C2AF1205BD120573
:1011DA00BD1205BDD2AF1205AD754C007888E6B4D4
:1011EA00030241C9120599788CE6C394015003029F
:1011FA0012C9E530C3940150030212C9207435C3E1
:10120A00E55C94FF50030212C9C2AF1205D2D2AFF5
:10121A001205A8C3E55C940150EFC2AF1205BD12D6
:10122A00059E1205BDD2AF1205A8C3E55C94FF4026
:10123A00E90217287F05D27F120FCB1205A8C2AF89
:10124A00C27F120FCBAE5CC3E55C947FD2AF40790C
:10125A00120594C2AF1205D2D2AFDFDA1102C3EE81
:10126A0094057897F61205AD1215CC1216AB7F0AC3
:10127A00D27F120FCB1205A8C2AFC27F120FCBAE1C
:10128A005CC3E55C947FD2AF50E4120594C2AF12FE
:10129A0005BD12059E1205BDD2AFDFD41102EE24A0
:1012AA00037896F61205AD1215CC1216DA1205A8B5
:1012BA00120FCBC3E55C94FF50024106021728C304
:1012CA00E55C954C4003855C4C1205A87801798849
:1012DA00E7B403027805C3E55C98400221E6C2AF91
:1012EA001205D21205D21205D2D2AF1205AD75304F
:1012FA0000E4F531F5320531E531F4703F05327815
:10130A009AE67819146012783214600D787D1460A8
:10131A000878FA146003753200C3E53298401D124A
:10132A000EC3120594153275310078998673C2AFCF
:10133A001205D2D2AF789886731205A812059EE5D7
:10134A002A700530740201E278012074027806C31B
:10135A00E55C9840A17888E6C3940360031205A867
:10136A00E52A70030210E2C2AF120EC3E4F522F5B9
:10137A0023F524F525F526F567D2AF7885E6C3333C
:10138A00F565E4F544F545F546F547F548F570F594
:10139A002CF52DF53775700875BB1E1205941208C9
:1013AA0061E5E820ECFBA8BDA9BEE97001F88871E7
:1013BA0012086575700875BB1E120F44C2AF7561BD
:1013CA00FF1208DD852261852262852263D2AF750C
:1013DA002201752401752501752601856069756AE2
:1013EA00017888E6B40307C27D307602D27DD268DE
:1013FA00D269753300120E1D120E4C1208FD120925
:10140A00041208FD1209041208FD120B7F1206AD20
:10141A00120C75120CBF120904120B6E306E0312F5
:10142A0006AE206703120800306703120847120C41
:10143A0075120CF4120904120B7F306E031206EABD
:10144A00120C75120D6B120904120B6E306E031218
:10145A000748120C75120D9A120904120B7F306E8E
:0D146A00031207A5120C75120E1D120904C5
:10147700120861120B6E120C75120E4C12086512CF
:10148700090430692F856461856462856069756ABE
:101497000179187A0CC3E53399400CC269D26A8A7C
:1014A700357561FF0214BBC3E55C94014003021468
:1014B70014021541306A1D206C1AE535147006C2F6
:1014C7006AD26B8114F535C3E55C940140030214BD
:1014D70014021541753600788279A4E76002780313
:1014E700C3E55F985054307404E52A604D7888E668
:1014F700B40317207D05207607A111307602A111CC
:10150700206C07D26C856461815378F0306C058557
:1015170064617820C3E5419850028114306C1BC286
:101527006CC27D307602D27DD26A753512856461D0
:1015370081140536E55C6002A144753600C2AF121E
:101547000EC37887E6FE7602120F447887EEF6E43C
:10155700F522F523F524F525F526F565752C007597
:101567002D00D2AF1205A8120EC378A4E66006D2EA
:1015770093D295D297307409C3E53694044002019B
:10158700E241FB901A0D782012160EE520B45A0C92
:10159700A312160EE520B4A5030215AC120ED8123D
:1015A70015CC0215CB901A0378807B0A12160EA36E
:1015B70008DBF9901A0F788C7B1912160EA308DB3B
:1015C700F9901A2822C2AF12164D121627901A0048
:1015D700740E121613A37406121613A3741512169B
:1015E70013901A0378807B0A121612A308DBF9906E
:1015F7001A0F788C7B19121612A308DBF9121660E2
:1016070012163E901A2822E493F622E6438F0153DE
:101617008FFD75EF0275B7A575B7F1F0538FFE22F1
:10162700438F02438F0175EF0275B7A575B7F19028
:101637001A0DF0538FFC22901A0D745AD113901A79
:101647000E74A5D113227A3079D07820901A40D120
:101657000EE520F709A3DAF7227A3079D0901A40FD
:10166700E7D11309A3DAF922AB74A875BB01027994
:1016770084BB02027985BB03027986BB0402799297
:10168700BB05027987BB060279A3BB0702799CBB1E
:1016970008027988BB09027989E8F7227C051205D7
:1016A700ADDCFB22C2AF1205BD1205C41205CB1279
:1016B70005D212059E1205BD1205C41205CB1205EF
:1016C700D212059E1205BD1205C41205CB1205D212
:1016D700D2AF22C2AF1205D21205CB1205C4120532
:1016E700BD12059E1205D21205CB1205C41205BD07
:1016F70012059E1205D21205CB1205C41205BDD2E2
:10170700AF22AE74AF75C2AF1205BD1205BD12058B
:10171700BD12059EDEF21205D212059EDFF8D2AF8A
:1017270022D1ABD1A3D1A37574017575017576006C
:10173700F1097C05AD5C1205ADC3ED955C70F5C391
:10174700E55C9401400AC3E55C94FF4032021764EC
:10175700D16FB1CCD1ABC2AF75EF12D1A3DCD50538
:1017670076C3E5769403500280C6D1A30575E57468
:101777001490009F93F808C3E57598500280AED186
:10178700A3D1A30574C3E574940A5002809C120E7A
:0A179700D8B1CCC2AF75EF12D1A398
:0319FD0002102FA6
:101A00000E0615FFFFFFFF0304070301015AA5019E
:101A1000FFFFFFFFFF03FFFFFF25D0FAFA04FF01DE
:091A2000007AFF0101000300FF40
:101A400023506C6174696E756D31353041232020EF
:101A500023424C48454C4923463331302320202033
:101A60002020202020202020202020202020202076
:101C0000C2AFC2D353D9BF7581C043B20343FF8073
:101C1000752438752503B1C975EF0275E24043F1AB
:101C20000853A4F775D4FFD2837DFA780379E67C54
:101C300010752200752300901DD67B0675249875BB
:101C400025013083028142208308D8FBD9F9DCF7D3
:101C500081B4308308D8FBD9F9DCF781B4B189E4C9
:101C600093A3C39A6004DDC381B4DBDBB17B600264
:101C7000812B7B08E493FAA3B15CDBF87A30B15C8A
:101C8000752200752300B17BEAFCEBFDC3ED94FEE9
:101C9000400EB17B8A278B28ED30E0048A828B834B
:101CA000B17B7AC270D8C3ED94FE601350CEBD00F4
:101CB00025EC60097520007521FF0200008100A855
:101CC00027A9280809D804D90281D3B17FEA89AAB3
:101CD000F281C50D81A0C3ED94035049EDA2E092BD
:101CE000007AC5C3E5829400E583941C50902000DF
:101CF00010438F02438F0175B7A575B7F1F030001F
:101D00001FA827A9280809438F01538FFDD804D99C
:101D100002A12089AAE275B7A575B7F1F0A3A10DBC
:101D2000538FFC817C7AC1BD030CE493A3FAB140CC
:101D3000DCF8B138817C817EAA22AB23B15CEBFA5E
:101D4000EA6222752608C3E52313F523E52213F57D
:101D50002250066323A0632201D526EAB1C9B1C986
:101D600075260AEAF4200102D283300102C283B14F
:101D7000C9C3134002C201D526EB22B17FEAFB2082
:101D80008302A17F308302A184752608AE24AF258B
:101D9000C3EF13FFEE13FEB1CDB1C9C3EA13308315
:101DA000024480FA30E703632201C3E52313F523DD
:101DB000E52213F52250066323A0632201D526D91C
:101DC000E52265236523F52222AE24AF250E0FDE22
:101DD000FEDFFCD20122424C48656C693437316326
:041DE000F3100601F5
:00000001FF
